:020000040000FA
:10000000FE28A2008316051083120930A3000310F6
:100010001020A20CA30B0828031410200314F928A5
:10002000031815280000051017280514172800309C
:10003000A1005B30A628A9004030A0004230A100FA
:100040000F30A400A501C320AA01210803192F28FD
:100050002A145C20FC3E031C2F28AA145C202003D9
:10006000AB00280F3728FF30A400A500422828083D
:10007000A500A401A600A7012B0A03194228A2008B
:10008000A301DD20A90B5B281508CF39A41B20385C
:10009000241B10380C389500250893008316051191
:1000A00083122B088316920083121208FC392A044B
:1000B00004389200F928F928A10CA00CA10CA00C7E
:1000C00008008320B400200821040319F928F32034
:1000D000A301A401340980208413FB202208A30774
:1000E00000083404031C34068000A40A0319A00A83
:1000F0000319A10F6D2834087D2884178004F9287E
:1001000084178005F928A8000530A8190530840057
:1001100000308A0028080739903E03188A0A8200B6
:100120000134023404340834103420344034803430
:10013000A301A200FF30A207031CA307031CF92898
:100140000330A100DF30A6209A28A101E83EA000DC
:10015000A109FC30031CAF28A0070318AC28A00796
:100160006400A10FAC282018B528A01CB9280000F5
:10017000B92808000038031DFF300405031DFF30B7
:10018000F928A501A4011030A600210DA40DA50D8C
:100190002208A4022308031C230FA5020318D72852
:1001A0002208A40723080318230FA5070310A00D96
:1001B000A10DA60BC5282008F9281030A800A10120
:1001C000A001A70CA60C031CEB282208A0072308FB
:1001D0000318230FA107A10CA00CA50CA40CA80BBD
:1001E000E1282408F928A009A109A00A0319A10AF5
:1001F00008008313031383126400080083169F0111
:1002000081131030950083121A3085000130C00030
:100210000230C1000A30BF00FF30BC000D300120A9
:100220000A3001200D3001200A3001204430012025
:1002300069300120743001206330012068300120D2
:10024000203001202F3001202030012043300120B8
:10025000723001206F300120733001207330012093
:10026000693001206E3001206730012020300120EC
:100270002F300120203001204D300120613001203D
:100280007230012073300120203001204C300120D9
:10029000693001206730012068300120743001206E
:1002A00020300120543001206530012073300120BE
:1002B000743001200A3001200D3001202830012047
:1002C000433001202930012020300120323001202C
:1002D0002D30012031300120323001202D3001201D
:1002E00032300120303001203130012038300120FF
:1002F000203001202D3001202030012064300120E9
:100300002E30012020300120623001206F3001208A
:10031000643001206E3001206130012072300120F4
:10032000203001202D3001202030012076300120A6
:10033000653001207230012020300120373001204B
:100340000D3001200A30012054300120723001208C
:1003500061300120693001206E30012045300120DC
:100360006C300120653001206330012074300120A1
:10037000723001206F3001206E3001206930012081
:1003800063300120733001202E30012063300120C2
:100390006F3001206D3001200D3001200A30012026
:1003A00003018519FF30B8000301051AFF30BA00B8
:1003B000380884003A08BA20BA00BB0064003A0842
:1003C0003B040319E5299501152A0301851DFF301A
:1003D000B8000301051AFF30BA00380884003A0853
:1003E000BA20BA00BB0064003A083B040319FA299A
:1003F00095018A2A0301051EFF30B8000301851903
:10040000FF30BA00380884003A08BA20031D2E2AAB
:10041000051583160511831285168316851283121E
:100420008514831685108312D029051183160511B2
:10043000831285168316851283120130A300F430CF
:1004400099208512831685128312051583160511CE
:1004500083120130A300F4309920D02905118316AE
:100460000511831285128316851283120130C30091
:100470004308A8002030A2004E30A30001301B200A
:100480000130A100F430A620C30F382AFF30C3008A
:10049000640001304302031C5D2A4308A800D030E9
:1004A000A2000730A30001301B200130A100F4306E
:1004B000A6200130C3020318482A0130C30064009B
:1004C0009C3043020318722A4308A8002030A2007F
:1004D0004E30A30001301B200130A100F430A620D3
:1004E000C30F5F2AAF30C300640001304302031C16
:1004F000892A4308A800D030A2000730A3000130A9
:100500001B200130A100F430A6200130C3020318E3
:10051000742AD0290D30BE000230BD009522023071
:10052000BE000D30BD009522D0293F08C2006400F6
:1005300042083C02031CB82A42083C02B800B90138
:10054000031CB9033F08B8070318B90A3808A2000A
:100550004008A000A1013E0861204208A200400816
:10056000A000A1013D0861204108C207031C972A91
:02057000080081
:020000040000FA
:02400E001C3F55
:00000001FF
